:020000040800F2
:100000007809002089010008B91B0008351A00088A
:10001000B51B000891020008D12200080000000072
:10002000000000000000000000000000E51E0008C5
:100030009502000800000000291C00083D1F000870
:10004000A3010008A3010008A3010008A301000800
:10005000A3010008A3010008A3010008A3010008F0
:10006000A3010008A3010008A3010008A3010008E0
:10007000A3010008A3010008A3010008A3010008D0
:10008000A3010008A3010008A3010008A3010008C0
:10009000A3010008A3010008A3010008A3010008B0
:1000A000A3010008A3010008A3010008A3010008A0
:1000B000A3010008A3010008A3010008A301000890
:1000C000A3010008A3010008A3010008A301000880
:1000D000A3010008A3010008A3010008A301000870
:1000E000A3010008A3010008A301000800F002F822
:1000F00000F03AF80AA090E8000C82448344AAF188
:100100000107DA4501D100F02FF8AFF2090EBAE885
:100110000F0013F0010F18BFFB1A43F0010318473B
:10012000C0220000E0220000103A24BF78C878C145
:10013000FAD8520724BF30C830C144BF04680C60ED
:10014000704700000023002400250026103A28BF35
:1001500078C1FBD8520728BF30C148BF0B60704739
:100160001FB51FBD10B510BD00F058F81146FFF7C0
:10017000F7FF02F0F7F800F076F803B4FFF7F2FFAC
:1001800003BC00F07DF8000009488047094800479B
:10019000FEE7FEE7FEE7FEE7FEE7FEE7FEE7FEE737
:1001A000FEE7FEE704480549054A064B7047000094
:1001B000A11F0008ED000008780300207809002046
:1001C00078050020780500204FF0000200B51346A6
:1001D00094469646203922BFA0E80C50A0E80C5067
:1001E000B1F12001BFF4F7AF090728BFA0E80C5018
:1001F00048BF0CC05DF804EB890028BF40F8042B11
:1002000008BF704748BF20F8022B11F0804F18BF7D
:1002100000F8012B7047704770477047754600F033
:100220002BF8AE4605006946534620F00700854688
:1002300018B020B5FFF7B6FFBDE820404FF000062C
:100240004FF000074FF000084FF0000BAC46ACE851
:10025000C009ACE8C009ACE8C009ACE8C00921F0AD
:1002600007018D46704710B50446AFF30080204665
:10027000BDE81040FFF781BF004870471000002024
:1002800001491820ABBEFEE72600020070470000BF
:10029000FFE7FEE77047000081B0EFF3108072B611
:1002A0000090FFE7FEE7000083B0019000208DF88A
:1002B0000300019890F8210002280DD0FFE7019972
:1002C00004208863FFE70199002081F82000FFE700
:1002D00001208DF80B0021E001980168086820F0EA
:1002E0000E00086001980168086820F001000860AD
:1002F0000198C16B026C012090404860FFE70199B2
:10030000012081F82100FFE70199002081F82000F9
:10031000FFE79DF803008DF80B00FFE79DF80B0049
:1003200003B0704781B000900098806B01B07047B7
:1003300090B00F900E9100200D900990FFE70E985D
:1003400000680D99C840002800F07F81FFE70D99F3
:10035000012088400C900E9800680C9908400B9082
:100360000B980C99884240F06C81FFE70E9840682A
:100370000590002851D0FFE7059801283AD0FFE703
:10038000059802283FD0FFE7059803285FD0FFE7D4
:100390000598112832D0FFE70598122838D0FFE7DA
:1003A00005980021C1F21101884236D0FFE7059877
:1003B0000021C1F2120188422FD0FFE705980021E9
:1003C000C1F22101884228D0FFE705980021C1F23F
:1003D0002201884221D0FFE705980021C1F23101B6
:1003E00088421AD0FFE705980021C1F23201884205
:1003F00013D02FE00E98C06809902CE00E98C068CA
:100400000430099027E00E98C0680830099022E077
:100410000E98C0680C3009901DE00E98806818B9DD
:10042000FFE70420099011E00E988068012806D1AA
:10043000FFE7082009900C980F99086105E0082053
:1004400009900C980F994861FFE7FFE703E000204F
:10045000099000E0FFE70B98FF2803D8FFE70F980B
:10046000049003E00F9804300490FFE7049808908C
:100470000B98FF2804D8FFE70D988000039006E052
:100480000D996FF01F0000EB81000390FFE70398C8
:10049000079008980068079A0F21914088430999AE
:1004A00091400843089908600E98C079C00600285A
:1004B00040F1C680FFE7FFE741F21800C4F20200F6
:1004C000016841F001010160006800F00100069040
:1004D0000698FFE70D9820F003000821C4F20101FF
:1004E00040580A900D9800F0030081000F2000FA98
:1004F00001F10A9888430A900F9840F60001C4F26F
:100500000101884203D1FFE70020029026E00F9806
:1005100040F60041C4F20101884203D1FFE7012007
:10052000019018E00F9841F20001C4F201018842E5
:1005300003D1FFE7022000900AE00F9941F2004248
:10054000C4F201020420914208BF03200090FFE79B
:1005500000980190FFE701980290FFE702980D993B
:1005600001F00301890000FA01F10A9808430A909A
:100570000A980D9921F003010822C4F20102885063
:100580000E988079C006002809D5FFE70B9A40F243
:100590000841C4F2010108681043086008E00B9AA2
:1005A00040F20841C4F20101086890430860FFE787
:1005B0000E9880798006002809D5FFE70B9A40F253
:1005C0000C41C4F2010108681043086008E00B9A6E
:1005D00040F20C41C4F20101086890430860FFE753
:1005E0000E9880798007002809D5FFE70B9A40F222
:1005F0000441C4F2010108681043086008E00B9A46
:1006000040F20441C4F20101086890430860FFE72A
:100610000E988079C00748B1FFE70B9A40F200417D
:10062000C4F2010108681043086008E00B9A40F228
:100630000041C4F20101086890430860FFE7FFE74A
:10064000FFE70D9801300D9079E610B0704700007B
:1006500040F27030C2F200000068704740F20400BF
:10066000C2F20000027840F27031C2F20001086864
:10067000104408607047000080B542F20001C4F2E7
:100680000201086840F010000860032000F08CF8B8
:100690000F2000F005F800F03BF8002080BD0000BE
:1006A00080B582B0009040F20000C2F20000006805
:1006B00040F20401C2F200010A784FF47A71B1FBF2
:1006C000F2F1B0FBF1F000F069FD20B1FFE701208D
:1006D0008DF8070018E000980F280DD8FFE7009963
:1006E0004FF0FF30002200F045F8009840F208017A
:1006F000C2F20001086003E001208DF8070003E06A
:1007000000208DF80700FFE79DF8070002B080BDCC
:1007100083B0FFE741F21800C4F20200016841F023
:1007200001010160006800F0010002900298FFE7FB
:10073000FFE741F21C00C4F20200016841F0805161
:100740000160006800F0805001900198FFE7FFE72A
:100750000421C4F2010108680090009820F0E060D4
:100760000090009840F08060009000980860FFE7DB
:1007700003B0704780B586B08DF8170004910392DE
:100780000020029001F0A6FD02909DF91700019053
:1007900002980499039A01F011FA0146019801F0B8
:1007A000A1FD06B080BD000080B582B00190019827
:1007B00001F0BAFD02B080BD80B584B00290019115
:1007C000029820B9FFE701208DF80F001BE1019886
:1007D00042F20001C4F20201096801F007018842F7
:1007E00016D9FFE742F20000C4F20200016821F0CE
:1007F0000701019A11430160006800F007000199A8
:10080000884204D0FFE701208DF80F00FBE0FFE7EE
:1008100002980078800700282AD5FFE70298007820
:100820004007002809D5FFE741F20401C4F20201A4
:10083000086840F4E0600860FFE70298007800076D
:10084000002809D5FFE741F20401C4F2020108685B
:1008500040F460500860FFE741F20401C4F2020175
:10086000086820F0F000029A926810430860FFE7E1
:1008700002980078C007002860D0FFE7029840681F
:1008800001280ED1FFE741F20000C4F20200006827
:100890008003002804D4FFE701208DF80F00B2E0A8
:1008A00021E00298406802280ED1FFE741F20000E3
:1008B000C4F2020000688001002804D4FFE7012090
:1008C0008DF80F009FE00DE041F20000C4F202003D
:1008D00000688007002804D4FFE701208DF80F008E
:1008E00091E0FFE7FFE741F20401C4F2020108686A
:1008F00020F00300029A526810430860FFF7A8FE38
:100900000090FFE741F20400C4F20200006800F02A
:100910000C0002994968B0EB810F0ED0FFE7FFF79A
:1009200097FE0099401A41F28931884204D3FFE7CB
:1009300003208DF80F0066E0E4E7FFE7019842F23C
:100940000001C4F20201096801F00701884216D2D1
:10095000FFE742F20000C4F20200016821F0070143
:10096000019A11430160006800F007000199884274
:1009700004D0FFE701208DF80F0044E0FFE7029864
:100980000078400700280CD5FFE741F20401C4F2CB
:100990000201086820F4E060029AD26810430860FF
:1009A000FFE702980078000700280DD5FFE741F225
:1009B0000401C4F20201086820F46050029A12692E
:1009C00040EAC2000860FFE700F04CF841F2040181
:1009D000C4F202010968C9B20A0942F29C31C0F6A8
:1009E0000001895CC84040F20001C2F200010860C9
:1009F00040F20800C2F200000068FFF751FE00203C
:100A00008DF80F00FFE79DF80F0004B080BD0000D7
:100A100040F20000C2F200000068704780B5FFF7A6
:100A2000F7FF41F20401C4F202010968C1F3022296
:100A300042F2AC31C0F60001895CC84080BD0000C4
:100A400080B5FFF7E5FF41F20401C4F20201096835
:100A5000C1F3C22242F2AC31C0F60001895CC84049
:100A600080BD000086B000200590049003900290A5
:100A7000019041F20400C4F202000068059005985C
:100A800000F00C000146009100283FD0FFE70098DD
:100A9000042804D0FFE70098082806D037E041F288
:100AA0000020C0F27A00019037E00598C0F383413E
:100AB00042F2B430C0F60000405C02909DF816008F
:100AC000C007C0B1FFE741F20400C4F202000068B1
:100AD000C0F3404142F2C430C0F60000405C0490D4
:100AE000029841F20021C0F27A0148430499B0FB18
:100AF000F1F0039007E0029840F60011C0F23D01CA
:100B000048430390FFE70398019006E0FFE741F2B6
:100B10000020C0F27A000190FFE7019806B070470C
:100B200080B586B00490049820B9FFE701208DF8C5
:100B300017002EE304980078C007002800F0AE806C
:100B4000FFE741F20400C4F20200006800F00C006C
:100B5000042813D0FFE741F20400C4F20200006849
:100B600000F00C0008281BD1FFE741F20400C4F29A
:100B700002000068C003002812D5FFE741F2000020
:100B8000C4F2020000688003002808D5FFE704983B
:100B9000406820B9FFE701208DF81700F9E27CE0FA
:100BA000FFE704984068B0F5803F09D1FFE741F2C4
:100BB0000001C4F20201086840F48030086032E0AD
:100BC0000498406868B9FFE741F20001C4F20201ED
:100BD000086820F480300860086820F480200860ED
:100BE00020E004984068B0F5A02F0DD1FFE741F256
:100BF0000001C4F20201086840F48020086008681F
:100C000040F4803008600CE041F20001C4F20201BF
:100C1000086820F480300860086820F480200860AC
:100C2000FFE7FFE7FFE7FFE704984068D0B1FFE781
:100C3000FFF70EFD0390FFE741F20000C4F202004F
:100C40000068800300280CD4FFE7FFF701FD03993B
:100C5000401A652804D3FFE703208DF8170098E2B7
:100C6000EAE719E0FFF7F4FC0390FFE741F2000028
:100C7000C4F202000068800300280CD5FFE7FFF7EC
:100C8000E7FC0399401A652804D3FFE703208DF899
:100C900017007EE2EAE7FFE7FFE7FFE70498007846
:100CA0008007002840F18D80FFE741F20400C4F284
:100CB0000200006810F00C0F13D0FFE741F20400AF
:100CC000C4F20200006800F00C00082829D1FFE7F8
:100CD00041F20400C4F202000068C003002820D4DE
:100CE000FFE741F20000C4F202000068800700281C
:100CF00009D5FFE704980069012804D0FFE7012027
:100D00008DF8170045E241F20001C4F202010868C3
:100D100020F0F800049A526940EAC2000860FFE738
:100D20004EE00498006958B3FFE70021C4F2422165
:100D300001200860FFF78CFC0390FFE741F2000000
:100D4000C4F202000068800700280CD4FFE7FFF718
:100D50007FFC0399401A032804D3FFE703208DF892
:100D6000170016E2EAE741F20001C4F20201086846
:100D700020F0F800049A526940EAC20008601EE0C0
:100D80000021C4F2422100200860FFF761FC0390BB
:100D9000FFE741F20000C4F202000068800700286B
:100DA0000CD5FFE7FFF754FC0399401A032804D33E
:100DB000FFE703208DF81700EBE1EAE7FFE7FFE725
:100DC000FFE7049800780007002848D5FFE704985B
:100DD000806918B3FFE740F28041C4F2422101204C
:100DE0000860FFF735FC0390FFE741F22400C4F2EE
:100DF00002000068800700280CD4FFE7FFF728FCFA
:100E00000399401A032804D3FFE703208DF8170045
:100E1000BFE1EAE7012000F009FF1FE040F2804156
:100E2000C4F2422100200860FFF712FC0390FFE7A4
:100E300041F22400C4F202000068800700280CD5AB
:100E4000FFE7FFF705FC0399401A032804D3FFE7E7
:100E500003208DF817009CE1EAE7FFE7FFE704981D
:100E600000784007002840F1D880FFE700208DF887
:100E7000070041F21C00C4F202000068C000002814
:100E800013D4FFE7FFE741F21C00C4F2020001683F
:100E900041F080510160006800F08050009000989F
:100EA000FFE701208DF80700FFE747F20000C4F2DA
:100EB00000000068C005002822D4FFE747F20001C7
:100EC000C4F20001086840F480700860FFF7C0FBBE
:100ED0000390FFE747F20000C4F200000068C0057D
:100EE00000280CD4FFE7FFF7B3FB0399401A6528ED
:100EF00004D3FFE703208DF817004AE1EAE7FFE794
:100F0000FFE70498C068012809D1FFE741F22001FA
:100F1000C4F20201086840F00100086031E0049862
:100F2000C06868B9FFE741F22001C4F20201086815
:100F300020F001000860086820F0040008601FE04D
:100F40000498C06805280DD1FFE741F22001C4F2E2
:100F50000201086840F004000860086840F00100E1
:100F600008600CE041F22001C4F20201086820F0A0
:100F700001000860086820F004000860FFE7FFE750
:100F8000FFE7FFE70498C068E0B1FFE7FFF760FB09
:100F90000390FFE741F22000C4F2020000688007DE
:100FA00000280ED4FFE7FFF753FB0399401A41F2E4
:100FB0008931884204D3FFE703208DF81700E8E069
:100FC000E8E71BE0FFF744FB0390FFE741F2200056
:100FD000C4F202000068800700280ED5FFE7FFF783
:100FE00037FB0399401A41F28931884204D3FFE765
:100FF00003208DF81700CCE0E8E7FFE79DF8070035
:10100000012809D1FFE741F21C01C4F2020108687E
:1010100020F080500860FFE7FFE70498C0690028CF
:1010200000F0B380FFE741F20400C4F20200006860
:1010300000F00C00082800F08280FFE70498C069E7
:1010400002285CD1FFE76021C4F242210020086041
:10105000FFF7FEFA0390FFE741F20000C4F202003E
:101060000068800100280CD5FFE7FFF7F1FA03992B
:10107000401A032804D3FFE703208DF8170088E007
:10108000EAE70498006AB0F5803F0CD1FFE741F22F
:101090000401C4F20201086820F40030049A926846
:1010A00010430860FFE741F20401C4F2020108683E
:1010B00020F47410049B1A6A5B6A1A431043086098
:1010C0006021C4F2422101200860FFF7C1FA0390B9
:1010D000FFE741F20000C4F202000068800100282E
:1010E0000CD4FFE7FFF7B4FA0399401A032804D39E
:1010F000FFE703208DF817004BE0EAE71EE06021D0
:10110000C4F2422100200860FFF7A2FA0390FFE733
:1011100041F20000C4F202000068800100280CD5F2
:10112000FFE7FFF795FA0399401A032804D3FFE776
:1011300003208DF817002CE0EAE7FFE724E004988D
:10114000C069012804D1FFE701208DF8170020E0D5
:1011500041F20400C4F2020000680290029800F418
:1011600080300499096A884208D1FFE7029800F4A8
:1011700070100499496A884204D0FFE701208DF875
:10118000170006E0FFE7FFE7FFE700208DF81700F4
:10119000FFE79DF8170006B080BD000080B582B063
:1011A0000190019800F0A0FE02B080BD85B00390D0
:1011B0000291FFE7039890F83C00012804D1FFE773
:1011C00002208DF813005BE00399012081F83C00B8
:1011D000FFE7FFE70399022081F83D0003980068CC
:1011E000406801900398006880680090019820F0A2
:1011F00070000190029801680198084301900198DD
:101200000399096848600398006842F60041C4F2F7
:101210000101884218D0FFE703980068B0F1804FC1
:1012200012D0FFE70398006840F20041C4F20001C9
:10123000884209D0FFE70398006840F60001C4F235
:10124000000188420ED1FFE7009820F08000009056
:101250000298416800980843009000980399096833
:101260008860FFE70399012081F83D00FFE70399BB
:10127000002081F83C00FFE700208DF81300FFE715
:101280009DF8130005B0704780B582B000900098BB
:1012900020B9FFE701208DF807003FE0009890F8A3
:1012A0003D0040B9FFE70099002081F83C0000981C
:1012B00000F038F8FFE70099022081F83D0000991E
:1012C00051F8040B00F06EFE0099012081F84600F1
:1012D000FFE70099012081F83E00009981F83F0066
:1012E000009981F84000009981F84100FFE7FFE78D
:1012F0000099012081F84200009981F8430000998B
:1013000081F84400009981F84500FFE70099012029
:1013100081F83D0000208DF80700FFE79DF80700E9
:1013200002B080BD82B001900198006840F2004197
:10133000C4F20001884210D1FFE7FFE741F21C0030
:10134000C4F20200016841F002010160006800F08F
:10135000020000900098FFE7FFE702B0704700002E
:1013600081B0009000980168C86820F00100C86052
:10137000FFE700980068006A41F21111084210D19D
:10138000FFE700980068006A40F24441084207D134
:10139000FFE700980168086820F001000860FFE797
:1013A000FFE7FFE70099012081F83D00002001B030
:1013B0007047000080B586B00490039100208DF83E
:1013C0000B00FFE7049890F83C00012804D1FFE7E8
:1013D00002208DF81700ABE00499012081F83C0051
:1013E000FFE7FFE70499022081F83D0004980068B8
:1013F00080680190019820F077000190019820F416
:101400007F400190019804990968886003980068FA
:101410000090002872D0FFE7009810286ED0FFE7F8
:10142000009820286AD0FFE70098302866D0FFE7B0
:101430000098402855D0FFE70098502837D0FFE7A4
:101440000098602840D0FFE7009870280BD0FFE795
:101450000098B0F5805F05D0FFE70098B0F5005F19
:1014600016D052E055E004980068039B5A689968CA
:10147000DB6800F01BFE049800688068019001980A
:1014800040F077000190019804990968886040E075
:1014900004980068039B5A689968DB6800F006FEB0
:1014A00004980168886840F48040886031E00498BE
:1014B0000068039A5168D26800F028FE049800681A
:1014C000502100F00DFE24E004980068039A516852
:1014D000D26800F043FE04980068602100F000FE2E
:1014E00017E004980068039A5168D26800F00EFE75
:1014F00004980068402100F0F3FD0AE004980068B9
:101500000399096800F0ECFD03E001208DF80B0061
:10151000FFE70499012081F83D00FFE704990020CE
:1015200081F83C00FFE79DF80B008DF81700FFE7FE
:101530009DF8170006B080BD80B588B00690FFE723
:10154000FFE70698006850E8030F20F4F07005905C
:10155000FFE705990698026842E803100028F0D1D9
:10156000FFE7FFE7FFE7FFE70698006850E8050F91
:1015700020F001000490FFE704990698026842E811
:1015800005100028F0D1FFE7FFE70698006B01285F
:1015900014D1FFE7FFE7FFE70698006850E8030F64
:1015A00020F010000390FFE703990698026842E8D4
:1015B00003100028F0D1FFE7FFE7FFE70698006877
:1015C00040690006002832D5FFE7FFE7FFE70698ED
:1015D000006850E8050F20F080000290FFE70299B4
:1015E0000698026842E805100028F0D1FFE7FFE7FF
:1015F0000698806BD0B1FFE70698816B00204863A6
:101600000698806BFEF750FE78B1FFE70698806B76
:10161000FEF788FE202807D1FFE7069910204864CE
:1016200003208DF81F004EE0FFE7FFE7FFE7069875
:10163000006840694006002832D5FFE7FFE7FFE772
:101640000698006850E8050F20F040000190FFE781
:1016500001990698026842E805100028F0D1FFE7DA
:10166000FFE70698C06BD0B1FFE70698C16B00207A
:1016700048630698C06BFEF717FE78B1FFE706983F
:10168000C06BFEF74FFE202807D1FFE70699102018
:10169000486403208DF81F0015E0FFE7FFE7FFE730
:1016A00006990020C8840699C88506994864069A58
:1016B000202182F84210069A82F8411006990863A8
:1016C0008DF81F00FFE79DF81F0008B080BD0000E7
:1016D00080B586B00490FFE7FFE70498006850E803
:1016E000030F20F490700390FFE7039904980268B9
:1016F00042E803100028F0D1FFE7FFE7FFE7FFE72C
:101700000498006850E8050F20F001000290FFE700
:1017100002990498026842E805100028F0D1FFE71A
:10172000FFE70498006B012814D1FFE7FFE7FFE70C
:101730000498006850E8030F20F010000190FFE7C4
:1017400001990498026842E803100028F0D1FFE7ED
:10175000FFE7FFE70498006840694006002832D59B
:10176000FFE7FFE7FFE70498006850E8050F20F067
:1017700040000090FFE700990498026842E80510D5
:101780000028F0D1FFE7FFE70498C06BD0B1FFE776
:101790000498C16B002048630498C06BFEF784FD79
:1017A00078B1FFE70498C06BFEF7BCFD202807D195
:1017B000FFE704991020486403208DF817000EE01D
:1017C000FFE7FFE7FFE704990020C885049A20217E
:1017D00082F84210049908638DF81700FFE79DF81E
:1017E000170006B080BD000080B584B00290FFE70E
:1017F000FFE70298006850E8030F20F0C000019056
:10180000FFE701990298026842E803100028F0D12E
:10181000FFE7FFE70298006840690006002832D51C
:10182000FFE7FFE7FFE70298006850E8050F20F0A8
:1018300080000090FFE700990298026842E80510D6
:101840000028F0D1FFE7FFE70298806BD0B1FFE7F7
:101850000298816B002048630298806BFEF724FD9C
:1018600078B1FFE70298806BFEF75CFD202807D176
:10187000FFE702991020486403208DF80F000CE068
:10188000FFE7FFE7FFE702990020C884029A2021C2
:1018900082F841108DF80F00FFE79DF80F0004B0AB
:1018A00080BD000080B582B00090009820B9FFE7AD
:1018B00001208DF8070040E00098806908B1FFE73B
:1018C00000E0FFE7009890F8410040B9FFE7009979
:1018D000002081F84000009800F034F8FFE70099FC
:1018E000242081F8410000980168C86820F4005065
:1018F000C860009800F05CFC00980168086920F45A
:101900009040086100980168486920F02A00486109
:1019100000980168C86840F40050C8600099002031
:101920004864009A202182F84110009A82F84210FF
:10193000009948638DF80700FFE79DF8070002B0A3
:1019400080BD000080B58AB0099000200890079003
:10195000069005900998006843F60001C4F2010161
:10196000884239D1FFE7FFE741F21800C4F20200D4
:10197000016841F480410160006800F480400490F7
:101980000498FFE7FFE741F21800C4F20200016883
:1019900041F004010160006800F004000390039826
:1019A000FFE74FF400700590022006900320089096
:1019B00040F60000C4F20100019005A90291FEF773
:1019C000B7FC019802994FF48062059200220692BA
:1019D0000792FEF7ADFCFFE70AB080BD80B584B08A
:1019E00002900191ADF80220029890F84200202860
:1019F00017D1FFE7019820B1FFE7BDF8020020B939
:101A0000FFE701208DF80F000FE002990020086326
:101A100002980199BDF8022000F028FC8DF80F0013
:101A200003E002208DF80F00FFE79DF80F0004B0DF
:101A300080BD0000FFE7FEE740F27001C2F2000146
:101A400042F2CF30C0F60000486042F2DF30C0F60C
:101A50000000C86042F2C632C0F600024A61C861A6
:101A6000486242F2D632C0F60002CA6248630720DA
:101A700008600120886009220A61886108620A22E0
:101A80008A6208637047000080B582B0FFF7D4FF18
:101A900040F2B820C2F2000001900121017041F231
:101AA0008832428301760221017740F22831C2F266
:101AB000000140F2E022C2F20002002300F082F9AD
:101AC000019981F8240002B080BD000081B0FFE7D9
:101AD00041F21800C4F20200016841F00401016003
:101AE000006800F0040000900098FFE701B0704724
:101AF00080B588B00021019107910691059104916C
:101B00000391029140F2E020C2F2000040F2004254
:101B1000C4F2000202600722426081604FF6FF7249
:101B2000C26001618161FFF7AFFB18B1FFE7FEF70B
:101B3000B3FBFFE74FF48050049040F2E020C2F284
:101B4000000004A9FFF736FC18B1FFE7FEF7A4FB7D
:101B5000FFE700200290039040F2E020C2F2000074
:101B600002A9FFF723FB18B1FFE7FEF795FBFFE79C
:101B700008B080BD80B582B040F22830C2F20000CB
:101B8000019043F60001C4F2010101604FF4E1311C
:101B9000416000218160C16001610C22426181616C
:101BA000C161FFF77FFE18B1FFE7FEF775FBFFE7A6
:101BB00002B080BDFFE7FEE7FFE7FEE788B00790D1
:101BC00006910592079800F0070004900498C0F170
:101BD0000700052803D3FFE70420019004E00498E0
:101BE000C0F107000190FFE70198039004980430CA
:101BF000062803D8FFE70020009003E0049803388C
:101C00000090FFE70098029006980399012202FADB
:101C100001F101390840029B984005999A40013A28
:101C20001140084308B070477047000082B001902F
:101C3000019840F20001C2F200010968C90844F6A7
:101C4000D352C1F26202A1FB0221890948430090EC
:101C5000FFE700BFFFE70098411E00910028F8D180
:101C6000FFE702B07047000080B584B003908DF8A4
:101C70000B1000208DF80A00039949690968486231
:101C80000398406901686FF0010008610398408B78
:101C900028B1FFE703984069FFF762FBFFE79DF873
:101CA0000B004007002844D4FFE79DF80B00800795
:101CB000002823D5FFE703980069FFF709FD8DF899
:101CC0000A00039991F8200000F0FB0081F8200041
:101CD000039991F8200000F0F70081F820000399A3
:101CE00091F8200000F0DF0081F82000039991F8BE
:101CF000200000F0FE0081F82000FFE79DF80B00B7
:101D0000C007A8B1FFE703980069FFF76DFD8DF8E4
:101D10000A00039991F8200000F0EF0081F82000FC
:101D2000039991F8200000F0BF0081F82000FFE740
:101D300042E003980069FFF7FFFB8DF80A000020DE
:101D40000190FFE70198B0F5817F0ADCFFE7039877
:101D50008168019A00208854FFE7019801300190C2
:101D6000F0E7039991F8200000F0FB0081F82000D3
:101D7000039991F8200000F0F70081F82000039902
:101D800091F8200000F0DF0081F82000039991F81D
:101D9000200000F0FE0081F82000039991F8200057
:101DA00000F0EF0081F82000039991F8200000F086
:101DB000BF0081F82000FFE70399032081F8240089
:101DC00004B080BD85B00390029101920093039806
:101DD00020B9FFE702208DF8130027E0029820B910
:101DE000FFE702208DF8130020E0029803990861B4
:101DF0000198039948610398007F20B9FFE702200A
:101E00008DF8130012E00398806838B9FFE7039952
:101E100040F2B410C2F20000886003E00098039919
:101E20008860FFE701208DF81300FFE79DF813009D
:101E300005B0704780B584B00290019100208DF804
:101E400003008DF80200029890F82000C008C00737
:101E500020B1FFE704208DF80F003FE0029991F8D0
:101E6000200040F0020081F82000029991F8200043
:101E700040F0080081F82000029991F8200000F05D
:101E8000DF0081F82000029991F8200000F0FE00A8
:101E900081F82000019802994860029881680069E1
:101EA0000722FFF79BFD8DF802009DF8020038B174
:101EB000FFE702980421FFF7D7FE8DF8030003E047
:101EC00001208DF80300FFE79DF80300029981F8D7
:101ED00024009DF803008DF80F00FFE79DF80F0028
:101EE00004B080BD7047000080B582B000900098BB
:101EF0000138B0F1807F03D3FFE70120019019E0A2
:101F0000009801384EF21401CEF2000108604FF043
:101F1000FF300F2100F0E6F94EF21801CEF2000179
:101F2000002008604EF21002CEF20002072111607C
:101F30000190FFE7019802B080BD000080B5FEF778
:101F40008DFB80BD80B590B006A800902821FEF7DB
:101F50003BF90098002105910491039102910191B0
:101F60000222069201220A9210220B920D91FEF794
:101F7000D7FD18B1FFE7FEF78FF9FFE70F200190BB
:101F80000021029103910491059101A8FEF714FC30
:101F900018B1FFE7FEF780F9FFE710B080BD000041
:101FA0007047000083B00290019102980068009091
:101FB000029842F60041C4F20101884215D0FFE7C1
:101FC0000298B0F1804F10D0FFE7029840F2004134
:101FD000C4F20001884208D0FFE7029840F60001F1
:101FE000C4F2000188420AD1FFE7009820F0700097
:101FF000009001984168009808430090FFE702981C
:1020000042F60041C4F20101884215D0FFE7029870
:10201000B0F1804F10D0FFE7029840F20041C4F2C7
:102020000001884208D0FFE7029840F60001C4F2A0
:10203000000188420AD1FFE7009820F44070009028
:102040000198C168009808430090FFE7009820F0CD
:10205000800001994969084300900098029908603E
:10206000019880680299C8620198006802998862A4
:10207000029842F60041C4F20101884205D1FFE70F
:102080000198006902990863FFE7029901204861FD
:1020900002980069C00730B1FFE70299086920F093
:1020A00001000861FFE703B07047000085B00490AD
:1020B000039102920193049880680090009820F4A4
:1020C0007F40009003980299019A41EA022101435E
:1020D00000980843009000980499886005B0704704
:1020E00083B002900191029880680090009820F0DF
:1020F0007000009001980099084340F0070000909C
:1021000000980299886003B07047000085B0049081
:10211000039102920498006A00900499086A20F0E2
:1021200001000862049880690190019820F0F00095
:1021300001900299019840EA01100190009820F066
:102140000A000090039900980843009001980499B0
:10215000886100980499086205B0704785B00490C2
:10216000039102920498006A00900499086A20F092
:1021700010000862049880690190019820F4704072
:1021800001900299019840EA01300190009820F0F6
:10219000A00000900399009840EA01100090019877
:1021A0000499886100980499086205B0704700009E
:1021B00080B584B0039003980068006920F4405013
:1021C000039A1168D26810430861039988680A6904
:1021D000496910430843029003980068C06841F2BF
:1021E0000C6188430299084303990968C860039801
:1021F0000068406920F44070039A116892691043A6
:1022000048610398006843F60001C4F20101884266
:1022100004D1FFE7FEF714FC019003E0FEF7FEFB9C
:102220000190FFE7019819214843039A1168526809
:102230009200B0FBF2FC48F21F52C5F2EB12ACFB6D
:1022400002304309642003FB10CC322000EB0C1059
:10225000A0FB0202F02000EA521000EB0310C2F3D0
:1022600043121044886004B080BD000083B0029027
:102270000191ADF80220019802998862BDF8020030
:1022800002998885BDF802000299C885029900204C
:1022900048640299222081F842000298006938B10E
:1022A000FFE702980168C86840F48070C860FFE7E3
:1022B00002980168486940F001004861029801688D
:1022C000C86840F02000C860002003B070470000DC
:1022D000FFE7FEE74EF60C50CEF200000068C0F3B8
:1022E0000220704782B08DF8070000919DF9070029
:1022F00000280AD4FFE7009800019DF907104EF26C
:102300000042CEF2000288540BE0009800019DF8D4
:10231000071001F00F014EF61452CEF2000288545D
:10232000FFE702B07047000083B00290029800F00F
:10233000070000904EF60C51CEF2000108680190A3
:1023400001984FF6FF02104001900198009A40EA70
:1023500002200022C0F2FA52104301900198086056
:1023600003B0704780B582B000200190FEF784F979
:10237000FFF7E8FDFFF7AAFBFFF7FCFBFFF7B8FB51
:10238000FFF782FB40F2B820C2F2000040F2A80141
:10239000C2F20001FFF74EFDFFE7FEE7000000007C
:1023A0000000000001020304060708090000000005
:1023B0000102030402030405060708090A0B0C0DB9
:1023C0000E0F101001025665722E20312E30004E75
:1023D000494F2D31320053544D33324631303300A2
:1023E0000024000800000020100000002801000860
:1023F00010240008100000206809000044010008B3
:1024000000127A000100000010000000000000002F
:04000005080000ED02
:00000001FF
